:100000008B018E010E1511288C00030E8D008B12B2
:1000100085019D01900191010D0E83008C0E0C0E47
:1000200009008316403081008501C33086008312A9
:100030000F3085003430860002210D2199000D21FA
:10004000031D2128AA30190203192A280221FF3092
:1000500024211C2897019D01900191018501F43014
:1000600024210D21060895008B17170882078F2879
:10007000942898289D28A0289D28A0289D28A0285D
:100080009D28A0289D28A0289D28A0289D28A0283C
:100090009D28A0289D28BE289D28C92894289828F6
:1000A0009D28AA289D28AA289D28AA289D28AA28F4
:1000B0009D28AA289D28AA289D28AA289D28AA28E4
:1000C0009D28BE289D28C928942898289D28B428B2
:1000D0009D28B4289D28B4289D28B4289D28B4289C
:1000E0009D28B4289D28B4289D28B4289D28BE2882
:1000F0009D28C928970147218E13191B8E170E13AF
:10010000191A0E171A08502190008E13991B8E177A
:100110000E13991A0E171B0850219100CD280E1DA1
:10012000CD280E11970ACD289C018615970ACD2857
:100130008618CD28061C970ACD288618970ACD2840
:100140008618CD28970A990C9913061CCD28991763
:100150009C0ACD288618CD28970A9A0C9A13061C5B
:10016000CD289A179C0ACD288618CD28970A9B0C73
:100170009B13061CCD289B179C0ACD288618CD28DA
:10018000970A1C18C62806180E14CD28061C0E1433
:10019000CD288618CD288611970A150896000608DE
:1001A000950016068039031935281D088207DF28B7
:1001B000EE28F72813080F3985009D013528951F73
:1001C000352810099200920A9001110893009101BC
:1001D000120E0F3985000E159D0A352812080F39A9
:1001E00085004E3081000B118B169D0A3528130EA9
:1001F0000F3985008B129D0A35280F309E009E0B0B
:10020000FF28080051309E009E0B04290729080092
:10021000861C082986180A2908009C018615061CD8
:1002200086180F29093097000821970B18291F29D4
:10023000980C9813061C142998179C0A1429082155
:10024000861102211808080098009C0186110221DD
:100250000611FD2086150830970086182D291818DC
:1002600033290611352906159C0A980C0821970B8D
:100270002F291C1806111C1C06150821061508211B
:10028000861C40298611061C432902210800191CDE
:10029000061619180612991C861699188612080057
:1002A0008F000E1F55298F098F0A8E1F8F1B8F01FC
:1002B0000F0803190800151B60298F0C8F138F0A74
:0C02C0000E1F64298F098F0A0F08080028
:084000000000010001000100B5
:02400E00F23F7F
:00000001FF
